:020000040000FA
:060000000A128A110C280F
:10000800FE00030EF0000A08F1000A168A11992F63
:100018000A128A110F288317C030FD000930FE002C
:10002800B630FF00903084000A168A11AD270A12F4
:100038008A118313C030FD000830FE007D30FF00B8
:10004800A03084000A168A11AD270A128A116E3070
:10005800FD001730FE004130FF00693084000A16A9
:100068008A11AD270A128A11C0308400D2300A16CC
:100078008A1163270A128A115730840069300A16D8
:100088008A116327FA01FB0183010A128A11A02D44
:10009800831203136008CC005F08CB006208CE000F
:1000A8006108CD006408D6006308D5005E08D0005A
:1000B8005D08CF006A08D2006908D1006C08D40036
:1000C8006B08D3001030C6004608F60002300A124A
:1000D8008A1597240A128A1153300A128A15842223
:1000E8000A128A11E92B0330C6004608F6000130CF
:1000F8000A128A1597240A128A113A300A128A15A6
:1001080084220A128A11063083120313C600460895
:10011800F60001300A128A1597240A128A113A3019
:100128000A128A1584220A128A11BC2B1030C600C2
:100138004608F60002300A128A1597240A128A1114
:1001480068300A128A1584220A128A11831203134C
:10015800861AE128073083120313C8005830C700F5
:100168005930C600C60BB628C70BB628C80BB62828
:10017800831203135F086004031DC7281730DF00CC
:100188000030E000CD280130DF020030031CE0031E
:10019800E002F601F60A01300A128A1597240A12BB
:1001A8008A11831203136008AD005F08AC000A12BD
:1001B8008A1587210A128A11D72B061AD72B0730DE
:1001C80083120313C8005830C7005930C600C60B45
:1001D800EB28C70BEB28C80BEB28831203135F0827
:1001E800013EC60060080318013E003EC70000300B
:1001F8004702183003194602031C0529DF01E001F4
:10020800CD280130DF070318E00A0030E007CD28C9
:100218001030C6004608F60002300A128A159724E4
:100228000A128A116D300A128A1584220A128A115A
:1002380083120313861A5529073083120313C80043
:100248005830C7005930C600C60B2829C70B2829C3
:10025800C80B28298312031361086204031D392976
:100268003B30E1000030E2003F290130E10200307C
:10027800031CE203E2020430C6004608F60001301F
:100288000A128A1597240A128A1183120313620824
:10029800AD006108AC000A128A1587210A128A117A
:1002A800D72B061AD72B073083120313C8005830F0
:1002B800C7005930C600C60B5F29C70B5F29C80B9A
:1002C8005F29831203136108013EC6006208031800
:1002D800013E003EC700003047023C300319460289
:1002E800031C7929E101E2013F290130E1070318E4
:1002F800E20A0030E2073F291030C6004608F6003F
:1003080002300A128A1597240A128A1173300A12C7
:100318008A1584220A128A1183120313861AB429B1
:10032800073083120313C8005830C7005930C6007D
:10033800C60B9C29C70B9C29C80B9C298312031345
:1003480063086404031DAD293B30E3000030E4007A
:10035800DE290130E3020030031CE403E402DE2955
:10036800061AD72B073083120313C8005830C7006A
:100378005930C600C60BBE29C70BBE29C80BBE29FB
:10038800831203136308013EC60064080318013E84
:10039800003EC700003047023C3003194602031CE8
:1003A800D829E301E401DE290130E3070318E40A50
:1003B8000030E4070730C6004608F60001300A128C
:1003C8008A1597240A128A11831203136408AD0050
:1003D8006308AC000A128A1587210A128A1183124F
:1003E800031364085606031DD72B63085506D72B3D
:1003F8001030C6004608F60002300A128A15972403
:100408000A128A1144300A128A1584220A128A11A1
:1004180083120313861A902A073083120313C80025
:100428005830C7005930C600C60B182AC70B182AFF
:10043800C80B182A831203136B08FF3EC6006C080A
:100448000318013EFF3EC70046084704031D402A23
:100458005E08B2005D08B1006A08B4006908B3001C
:100468000A128A11C5270A128A1183120313320845
:10047800EC003108EB00462A0130EB020030031C87
:10048800EC03EC020230C6004608F60002300A12FD
:100498008A1597240A128A11831203135E08AD0085
:1004A8005D08AC006A08AF006908AE006C08B100CE
:1004B8006B08B0000A128A156C260A128A11831278
:1004C80003132D08BD002C08BC000A168A118B27BF
:1004D8000A128A1183120313BF000030C0000A12E7
:1004E8008A1538230A128A11063083120313C600AC
:1004F8004608F60002300A128A1597240A128A1151
:10050800831203136C08AD006B08AC000A128A153D
:1005180087210A128A11D72B061AD72B0730831284
:100528000313C8005830C7005930C600C60B9A2AB2
:10053800C70B9A2AC80B9A2A831203136B08013E29
:10054800C6006C080318013E003EC7005E08B200F2
:100558005D08B1006A08B4006908B3000A128A117C
:10056800C5270A128A118312031347083202031D92
:10057800BF2A460831020318C62A0130EB000030B2
:10058800EC00462A0130EB070318EC0A0030EC07B0
:10059800462A1030C6004608F60002300A128A15AC
:1005A80097240A128A114D300A128A1584220A12D7
:1005B8008A1183120313861A1B2B07308312031325
:1005C800C8005830C7005930C600C60BE92AC70B07
:1005D800E92AC80BE92A831203136908FF3EC600FB
:1005E8006A080318013EFF3EC70046084704031D7A
:1005F800FF2A0C303D2B0130E9020030031CEA03CE
:10060800EA020930C6004608F60002300A128A15C6
:1006180097240A128A11831203136A08AD00690825
:10062800AC000A128A1587210A128A11D72B061ADA
:10063800D72B073083120313C8005830C70059302E
:10064800C600C60B252BC70B252BC80B252B8312E1
:1006580003136908013EC6006A080318013E003EFC
:10066800C700003047020D3003194602031C412B16
:100678000130E9000030EA00052B0130E9070318D2
:10068800EA0A0030EA07052B1030C6004608F600D3
:1006980002300A128A1597240A128A1159300A124E
:1006A8008A1584220A128A1183120313861A912B3F
:1006B800073083120313C8005830C7005930C600EA
:1006C800C60B642BC70B642BC80B642B8312031354
:1006D8005D085E04031D752B6330DD000030DE000D
:1006E8007B2B0130DD020030031CDE03DE020E30FE
:1006F800C6004608F60002300A128A1597240A1224
:100708008A11831203135E08AD005D08AC000A125B
:100718008A1587210A128A11D72B061AD72B073078
:1007280083120313C8005830C7005930C600C60BDF
:100738009B2BC70B9B2BC80B9B2B831203135D08AA
:10074800013EC6005E080318013E003EC7000030A7
:100758004702643003194602031CB52BDD01DE0194
:100768007B2B0130DD070318DE0A0030DE077B2B08
:10077800831203136608003A0319C32BD72B6508A5
:10078800013A03199A28033A03190C29013A031963
:100798008029073A0319482B013A0319CD2A033A4D
:1007A8000319FC29D72B831203130619F12B0730E1
:1007B80083120313C8005830C7005930C600C60B4F
:1007C800E32BC70BE32BC80BE32B01308312031376
:1007D800E5070318E60A0030E6076508660403190A
:1007E800FC2B00306602073003196502031C7728CA
:1007F80000306602073003196502031C0800103038
:10080800C6004608F60002300A128A1597240A1212
:100818008A11103083120313BF008030C0000A12FF
:100828008A1538230A128A1183120313E501E60197
:1008380060084C06031D222C5F084B06031D4C2C38
:1008480062084E06031D2A2C61084D06031D4C2C18
:1008580064085606031D322C63085506031D4C2CEC
:100868005E085006031D3A2C5D084F06031D4C2CEC
:100878006A085206031D422C69085106031D4C2CB8
:100888006C085406031D4A2C6B085306031908000C
:100898000A128A1542250A128A11831203135E0866
:1008A800AD005D08AC006A08AF006908AE006C08CE
:1008B800B1006B08B0000A128A156C260A128A1158
:1008C800831203132D08BD002C08BC000A128A15D8
:1008D80031210A128A110A128A15A2250800F60186
:1008E800F60A01300A128A1597240A128A1183120D
:1008F80003136008AD005F08AC000A128A1587214F
:100908000A128A11043083120313C6004608F6003F
:1009180001300A128A1597240A128A1183120313C6
:100928006208AD006108AC000A128A1587210A1214
:100938008A11073083120313C6004608F6000130F7
:100948000A128A1597240A128A118312031364085B
:10095800AD006308AC000A128A1587210A128A11B1
:10096800063083120313C6004608F60002300A1246
:100978008A1597240A128A11831203136C08AD0092
:100988006B08AC000A128A1587210A128A110930ED
:1009980083120313C6004608F60002300A128A15AD
:1009A80097240A128A11831203136A08AD00690892
:1009B800AC000A128A1587210A128A110C30831298
:1009C8000313C6004608F60002300A128A15972457
:1009D8000A128A11143083120313AC000030AD00E0
:1009E8000A128A1587210A128A110E3083120313FC
:1009F800C6004608F60002300A128A1597240A1221
:100A08008A11831203135E08AD005D08AC000A1258
:100A18008A1587210A128A11023083120313C6002D
:100A28004608F60002300A128A1597240A128A111B
:100A380083160313230883120313BD0083160313BD
:100A4800220883120313BC000A168A118B270A1284
:100A58008A1183120313BF000030C0000A128A15DE
:100A680038230A128A110A3083120313C600460873
:100A7800F60001300A128A1597240A128A11831285
:100A880003136D080A128A1584220A128A11831226
:100A980003135808AD005708AC000A128A158721BD
:100AA8000A128A110E3083120313C6004608F60094
:100AB80001300A128A1597240A128A110A30831201
:100AC8000313A0000030A1005A08A3005908A2008F
:100AD8000A128A15FA220A128A11831203132008AD
:100AE800303E0A128A1584220A128A1183120313CD
:100AF80061086204031D8D2D63086404031D8D2D98
:100B08000230F2000030F3000A128A1503240A1298
:100B18008A111E308312031361066204031D080044
:100B280063086404031D08000130F2000030F3007C
:100B38000A128A15032408008316031305140615E0
:100B4800061686168B1381130B168B1787018312D3
:100B58000313870183160313880183120313880183
:100B68000030F5000130F4008630F300A030F200C8
:100B78000A168A11BA270A128A110A168A117F27B9
:100B88000A128A110A128A1503260A128A110030DB
:100B9800F700F8000A128A15BE200A128A110A12F2
:100BA8008A1579230A128A110A128A15BC230A1295
:100BB8008A11403083120313AA000030AB000A12D6
:100BC8008A1507210A128A110330F7000030F8004D
:100BD8000A128A15BE200A128A11831603135008B6
:100BE80051040319462E0330D2005208F600013092
:100BF8000A128A1597240A128A113A300A128A159B
:100C080084220A128A11063083160313D20052086E
:100C1800F60001300A128A1597240A128A113A300E
:100C28000A128A1584220A128A110A128A151027B2
:100C38000A128A110A128A11C8260A128A110A127D
:100C48008A155D200A128A110A128A154E220A1282
:100C58008A110A128A1173240A128A11831603133D
:100C6800D001D1010D3083160313D400AF30D30067
:100C7800B530D200D20B3E2ED30B3E2ED40B3E2ED7
:100C8800452E682E0330D2005208F60001300A12B1
:100C98008A1597240A128A1120300A128A1584228A
:100CA8000A128A11063083160313D2005208F6007E
:100CB80001300A128A1597240A128A1120300A1262
:100CC8008A1584220A128A118312031306197F2EA9
:100CD800073083160313D4005830D3005930D2009C
:100CE800D20B742ED30B742ED40B742E0A128A11C5
:100CF8004C200A128A110030F200F3000A128A15F9
:100D080040200A128A117308FB007208FA007B0857
:100D180083160313D3007A08D2005308D200D301F4
:100D2800831203136808831603135306031DA22EA8
:100D38008312031367088316031352060319F12D50
:100D48007B08D3007A08D2005308D200D301520896
:100D5800F7005308F8000A128A15BE200A128A11F1
:100D68007B0883160313D3007A08D2005308D200F5
:100D7800D301520883120313E700831603135308A1
:100D880083120313E800F12D0A168A114D270A125F
:100D98008A11D03083120313A8000030A9000A1664
:100DA8008A115B270A128A11073083120313A800DD
:100DB8000030A9000A168A115B270A128A110A163E
:100DC8008A1146270A128A11D13083120313A80008
:100DD8000030A9000A168A115B270A128A1101300D
:100DE800F2000030F3000A128A155B210A128A11F8
:100DF8007308F9007208F8000A128A15E0200A122E
:100E08008A11790883160313CF007808CE000130C1
:100E1800F2000030F3000A128A155B210A128A11C7
:100E28007308F9007208F8000A128A15E0200A12FD
:100E38008A11790883160313CD007808CC00013095
:100E4800F2000030F3000A128A155B210A128A1197
:100E58007308F9007208F8000A128A15E0200A12CD
:100E68008A11790883160313CB007808CA00013069
:100E7800F2000030F3000A128A155B210A128A1167
:100E88000130F2000030F3000A128A155B210A12C1
:100E98008A117308F9007208F8000A128A15E0200E
:100EA8000A128A11790883160313C9007808C80042
:100EB8000130F2000030F3000A128A155B210A1291
:100EC8008A117308F9007208F8000A128A15E020DE
:100ED8000A128A11790883160313C7007808C60016
:100EE8000130F2000030F3000A128A155B210A1261
:100EF8008A110130F2000030F3000A128A155B21D2
:100F08000A128A11730883120313DC007208DB00CB
:100F18000130F2000030F3000A128A155B210A1230
:100F28008A11730883160313C5007208C4000130C0
:100F3800F2000030F3000A128A155B210A128A11A6
:100F48000130F2000030F3000A128A155B210A1200
:100F58008A11730883120313D8007208D70000306F
:100F6800F200F3000A128A155B210A128A1173082B
:100F780083120313DA007208D9000A168A1154275B
:100F88000800023083120313330634040319ED2FCB
:100F98000730A7000030A8003308FF3EA900340836
:100FA8000318013EFF3EAA000A128A15E621013005
:100FB800831203132705B50000302805B6001F303B
:100FC800B70035083702B10036090318013EB200F0
:100FD80008003208AD003108AC000A128A15BD229B
:100FE800831203132C081C3EB1002D080318013E80
:060FF800003EB2000800FB
:10100000FF1B0A2883137F1883170008840A03191B
:10101000FF0A080008308A000408840A82070034A6
:1010200020346434643464342034443444342F34FD
:101030004D344D342F3443344334593459342034EF
:101040000034483448343A346D346D343A347334AF
:10105000733420342D34503450342E345034003412
:101060004434653473346B34203443346C346F341B
:0C10700063346B340034563431340034E7
:101080007208F400F40DF40DF40D831203131F081D
:101090007406C73974069F001F140830F400F40B5F
:1010A0004F28831203131F151F1954281E08F3001D
:1010B000831603131E08F200080001308312031385
:1010C0005B0583160313C2000030831203135C0513
:1010D00083160313C300831203135C08F3005B0839
:1010E000F2000310F30CF20C0130720583160313A7
:1010F000C00000307305C10008001434003401340E
:101100000034533475346E3400344D346F346E34DF
:1011100000345434753465340034573465346434E1
:1011200000345434683475340034463472346934CD
:1011300000345334613474340034F601F701721C06
:10114000A7287408F6070318F70A7508F70701308F
:101150000310F40DF50DFF3E031DA8280130031008
:10116000F30CF20CFF3E031DAF2872087304031D3D
:101170009F287708F3007608F200080003300A166B
:101180008A11E6270A128A15483083120313A10038
:101190006B30A000A00BCA28A10BCA28CF280330AF
:1011A0000A168A11E6270A128A1502300A168A11CF
:1011B000E6270A128A1577080A128A15842208007F
:1011C0000F30780583120313A00000307905A100C9
:1011D000780E0F39F200790EF039F204790E0F39DA
:1011E000F300F030F31D0030F3040A30F400003057
:1011F000F5000A128A159D20831203132008720736
:10120000F80021080318210A7307F90008000A16DC
:101210008A114D270A128A15D03083120313A800B1
:101220000030A9000A168A115B270A128A150E30AF
:1012300083120313A8000030A9000A168A115B2745
:101240000A128A15831203132B08A9002A08A80082
:101250000A168A115B270A128A150A168A11542760
:1012600008000A168A114D270A128A15D0308312F7
:101270000313A8000030A9000A168A115B270A127E
:101280008A15033083120313A8000030A9000A1640
:101290008A115B270A128A15831203133D08A900DD
:1012A0003C08A8000A168A115B270A128A150A163A
:1012B0008A11542708000A168A116B270A128A1508
:1012C0008316031391150A168A116B270A128A15C1
:1012D000831203131308F400F5017408F60075086F
:1012E000F7000A168A116B270A128A15720873040E
:1012F000031D7E2983160313911681298316031378
:10130000911211167708F3007608F20008000A30EF
:1013100083120313A0000030A1002D08A3002C08A5
:10132000A2000A128A15FA220A128A1583120313DE
:101330002008303E0A128A1584220A128A150A30C1
:1013400083120313A7000030A8002D08AA002C0860
:10135000A9000A128A15E6210A128A1583120313BC
:101360002708303E0A128A15842208004A34613464
:101370006E34003446346534623400344D346134A4
:101380007234003441347034723400344D3461347A
:10139000793400344A3475346E3400344A34753448
:1013A0006C3400344134753467340034533465345C
:1013B000703400344F346334743400344E346F343A
:1013C00076340034443465346334003483120313B8
:1013D000270828040319152AAB01AB0AA81BFC290E
:1013E00001300310A70DA80DFF3E031DF1290130A8
:1013F000F9007908AB07EE2928082A02031D022A02
:1014000027082902031C0A2A2708A9022808031C06
:10141000AA03AA0201300310A80CA70CFF3E031D6B
:101420000B2A0130AB02031DFC292A08A800290859
:10143000A70008000A30F2000030F3008312031303
:101440002508F5002408F4000A128A15E7240A1278
:101450008A15720883120313A6007308A700A60E4C
:10146000A70EF030A70526080F39A704F030A6050F
:101470000A30F2000030F3002508F5002408F400DB
:101480000A128A154C247208831203132607A4003B
:1014900073080318730A2707A500080083120313B3
:1014A000D81F672AFF30F200FF30F3005808F5001C
:1014B0005708F4000A128A159D200A128A1573082B
:1014C00083120313D8007208D7002D30682A2B30FE
:1014D000F8007808ED0006300310DA0CD90CFF3E56
:1014E000031D6C2A1930F2000030F3005A08F50091
:1014F0005908F4000A128A159D20730883120313F9
:10150000DA007208D9000800F60076080F39F300F7
:101510007308F4007608F039F3007308F5008312BD
:10152000031308157508F30004300310F30CFF3E95
:10153000031D952A73080A168A11CC270A128A15E8
:101540008312031388154230F300F30BA52A000021
:1015500083120313881174080A168A11CC270A1201
:101560008A158312031388154230F300F30BB62A51
:101570000000831203138811080083120313B001C3
:1015800003305D05AE0000305E05AF002E082F046D
:10159000031DF22A6430A7000030A8005E08AA00EC
:1015A0005D08A9000A128A15E6210A128A1583121B
:1015B000031327082804031DF02A9030A7000130E8
:1015C000A8005E08AA005D08A9000A128A15E62193
:1015D0000A128A158312031327082804031DF22A0E
:1015E000B001B00A3008AE00AF012E08AC002F08E1
:1015F000AD00080083120313A501A60120082104F1
:101600000319332BA401A40AA11B122B01300310D0
:10161000A00DA10DFF3E031D072B0130F800780837
:10162000A407042B01300310A50DA60DFF3E031DDA
:10163000132B21082302031D1F2B20082202031C49
:10164000282B2008A2022108031CA303A3022514AF
:1016500001300310A10CA00CFF3E031D292B01300B
:10166000A402031D122B2608A1002508A0000800D3
:1016700083120313C401C50144083F07C200400898
:10168000C1000318C10AC41BC1038312031341081C
:10169000C3004308FF00420884000A128A15002094
:1016A0000A128A15003A0319080044083F07C200CD
:1016B0004008C1000318C10AC41BC10383120313ED
:1016C0004108C3004308FF00420884000A128A153B
:1016D00000200A128A150A128A1584220A128A1513
:1016E000013083120313C4070318C50A0030C5076D
:1016F0003C2B0A168A1174270A128A1504308312A9
:101700000313C6004608F60001300A128A15972412
:101710000A128A15213083120313BF008030C000E3
:101720000A128A1538230A128A150F3083120313FE
:10173000C6004608F60002300A128A1597240A12DB
:101740008A152C3083120313BF008030C0000A12A8
:101750008A1538230A128A151A3083120313C80017
:101760005E30C7006D30C600C60BB42BC70BB42B60
:10177000C80BB42BBB2B08000A168A1174270A1257
:101780008A15F601F60A01300A128A1597240A1200
:101790008A15123083120313BF008030C0000A1272
:1017A0008A1538230A128A15DF300A128A15842214
:1017B0000A128A1543300A128A1584220A128A15DF
:1017C000F601F60A02300A128A1597240A128A15BF
:1017D000013083120313BF008030C0000A128A1543
:1017E00038230A128A151A3083120313C8005E3098
:1017F000C7006D30C600C60BFB2BC70BFB2BC80BFD
:10180000FB2B022C080083120313A001A101730813
:101810002102031D0D2C7208200203180800A201EA
:10182000A3018312031388140330F5006E30F40013
:10183000F40B182CF50B182C831203138810D030DE
:10184000F400F40B212C013083120313A2070318B8
:10185000A30A0030A3072308803AFF0080307F02EC
:10186000031D342CFA302202031C112C0D30F6001B
:10187000AF30F500B630F400F40B3C2CF50B3C2CEB
:10188000F60B3C2C0000013083120313A007031851
:10189000A10A0030A107072CF801F51F562CF40906
:1018A000F509F40A0319F50AF801F80AF31F5D2C8B
:1018B000F209F309F20A0319F30A7208730403190F
:1018C0008A2CF701F70AF31B712C01300310F20D7B
:1018D000F30DFF3E031D662C0130F6007608F70776
:1018E000632C73087502031D772C72087402031CA5
:1018F0007F2C7208F4027308031CF503F502013013
:101900000310F30CF20CFF3E031D802C0130F70294
:10191000031D712C78080319922CF409F509F40AB7
:101920000319F50A7508F3007408F2000800831221
:101930000313A0002003031DC02C76087F3EF70090
:101940007708A3002308F70004300310F70CFF3ECC
:10195000031DA52C7708F8007808A10023080F398B
:10196000F7007708A20021080A168A11E6270A1252
:101970008A158312031322080A168A11E627080023
:1019800002302006031D08007608BF3EF7007708E6
:10199000A3002308F70004300310F70CFF3E031DDB
:1019A000CC2C7708F8007808A10023080F39F7003D
:1019B0007708A20021080A168A11E6270A128A155A
:1019C0008312031322080A168A11E62708008312DD
:1019D0000313A101F31FF32CF209F309F20A03190F
:1019E000F30AA101A10AF51FFE2CF409F509F40A76
:1019F0000319F50A0130F6007608A106A201A30139
:101A0000720873040319352DA001A00AF31B142DCD
:101A100001300310F20DF30DFF3E031D092D0130BF
:101A2000F6007608A007062D01300310A20DA30DC5
:101A3000FF3E031D152D73087502031D212D72082D
:101A40007402031C2A2D7208F4027308031CF503A8
:101A5000F502221401300310F30CF20CFF3E031DBB
:101A60002B2D0130A002031D142D210803193D2D3B
:101A7000A209A309A20A0319A30A2308F300220852
:101A8000F20008000A168A114D270A128A15D03072
:101A900083120313A8000030A9000A168A115B27DD
:101AA0000A128A15003083120313A800A9000A162F
:101AB0008A115B270A128A15831203136408A50092
:101AC0006308A4000A128A151A220A128A158312C0
:101AD00003132508A9002408A8000A168A115B2709
:101AE0000A128A15831203136208A5006108A40074
:101AF0000A128A151A220A128A158312031325085C
:101B0000A9002408A8000A168A115B270A128A1560
:101B1000831203136008A5005F08A4000A128A1547
:101B20001A220A128A15831203132508A900240811
:101B3000A8000A168A115B270A128A150A168A114A
:101B4000542708000A168A114D270A128A15D03028
:101B500083120313A8000030A9000A168A115B271C
:101B60000A128A15043083120313A8000030A9005A
:101B70000A168A115B270A128A15831203136C084E
:101B8000A5006B08A4000A128A151A220A128A15E7
:101B9000831203132508A9002408A8000A168A1135
:101BA0005B270A128A15831203136A08A5006908C5
:101BB000A4000A128A151A220A128A158312031324
:101BC0002508A9002408A8000A168A115B270A1212
:101BD0008A15831203135E08A5005D08A4000A128B
:101BE0008A151A220A128A15831203132508A900DE
:101BF0002408A8000A168A115B270A128A150A16F9
:101C00008A115427080000300A168A11CC270A12BC
:101C10008A15823083120313A300DD30A200A20BC9
:101C20000F2EA30B0F2E03300A168A11E6270A1275
:101C30008A15213083120313A3007530A200A20B72
:101C40001F2EA30B1F2E242E03300A168A11E627FF
:101C50000A128A15483083120313A3006B30A200C6
:101C6000A20B302EA30B302E352E03300A168A110C
:101C7000E6270A128A1502300A168A11E6270A1286
:101C80008A150030F700F8000A128A15BE200A12E1
:101C90008A1502300A168A11E6270A128A150830B8
:101CA0000A168A11E6270A128A1500300A168A11C6
:101CB000E6270A128A150C300A168A11E6270A123C
:101CC0008A1500300A168A11E6270A128A1506308C
:101CD0000A168A11E62708000030831203132F0228
:101CE000033003192E02031C842E2C08FE3EB20082
:101CF0002D080318013EFF3EB3003208B007031859
:101D0000B10A3308B107902E2C08B0070318B10AA6
:101D10002D08B1070130AC020030031CAD03AD0249
:101D20000730A7000030A8002D08B3002C08B2002F
:101D30000310B30CB20C0310B30CB20C0930A000AA
:101D40000030A1002F08F3002E08F2001730F40035
:101D50000030F5000A128A159D200A128A157308B0
:101D600083120313A3007208A2000A128A15FA2232
:101D70000A128A158312031332082007B4003308AD
:101D80000318330A2107B5009030A0000130A100EC
:101D90002D08A3002C08A2000A128A15FA220A12A2
:101DA0008A158312031320083407B600210803188C
:101DB000210A3507B7006430A0000030A1002D08CB
:101DC000A3002C08A2000A128A15FA220A128A1508
:101DD0008312031320083602B8002108031C210ACD
:101DE0003702B90030083807BA0031080318310A41
:101DF0003907BB003A08043EA9003B080318013E1E
:101E0000003EAA000A128A15E6218312031327084E
:101E1000013EAC0028080318013E003EAD0008005A
:101E20000A168A114D270A128A15D030831203131D
:101E3000A8000030A9000A168A115B270A128A1529
:101E4000003083120313A800A9000A168A115B2729
:101E50000A128A150A168A1154270A128A150A16B6
:101E60008A114D270A128A15D13083120313A80054
:101E70000030A9000A168A115B270A128A15013060
:101E8000F2000030F3000A128A155B210A128A154B
:101E90007308F9007208F8000A128A15E0200A1285
:101EA0008A15790883120313E4007808E3000130EF
:101EB000F2000030F3000A128A155B210A128A151B
:101EC0007308F9007208F8000A128A15E0200A1255
:101ED0008A15790883120313E2007808E1000130C3
:101EE000F2000030F3000A128A155B210A128A15EB
:101EF0007308F9007208F8000A128A15E0200A1225
:101F00008A15790883120313E0007808DF00013096
:101F1000F2000030F3000A128A155B210A128A15BA
:101F2000730883160313A3007208A2000130F200A5
:101F30000030F3000A128A155B210A128A15730811
:101F4000F9007208F8000A128A15E0200A128A15B0
:101F5000790883120313EC007808EB000130F200DB
:101F60000030F3000A128A155B210A128A157308E1
:101F7000F9007208F8000A128A15E0200A128A1580
:101F8000790883120313EA007808E9000130F200AF
:101F90000030F3000A128A155B210A128A157308B1
:101FA000F9007208F8000A128A15E0200A128A1550
:101FB000790883120313DE007808DD000A168A11FF
:101FC00054270A128A150A168A114D270A128A15F1
:101FD000D13083120313A8000030A9000A168A1119
:101FE0005B270A128A150130F2000030F3000A1252
:101FF0008A155B210A128A150A168A1154270800CD
:102E8200013400340134003420340A168A116B27CD
:102E920083160313911408000A168A116B278316EE
:102EA2000313111408000A168A116B2783160313E1
:102EB200111508000A168A116B27831203132808BA
:102EC2009300080064008001840A04060319003498
:102ED2000406642F8316031311081F39031D6B2F79
:102EE200141D08006B2F00300A168A11E6270A16F5
:102EF2008A1101300A168A11E62708008312031389
:102F02009F011F139F17831603139F171F119F10F3
:102F12001F100800831203133C08BE000130031087
:102F2200BE0DFF3E031D902F03103E0DA03E080074
:102F32008B1CA22F013083160313D0000030D10066
:102F42008B1071088A00700E8300FE0E7E0E09003F
:102F52007E088A007F088200A9270A168A1180004B
:102F6200840A04087D0603190034FF0A0319FE0AC5
:102F7200AD2F831603138715071628308312031308
:102F82009400831603139101313093009417831236
:102F9200031314120800F200721CD32F83120313BE
:102FA2000816D62F831203130812F21CDA2F881682
:102FB200DB2F8812721DDF2F0817E02F0813F21D76
:102FC200E42F8817080088130800F5008312031302
:102FD200081175080A168A11CC270A168A1183125B
:102FE200031388151A30F400F830F300F30BF72FAF
:0E2FF200F40BF72F0000831203138811080060
:02400E00723FFF
:00000001FF
